:1000000000308A00692800000A108A100A1182074D
:1000100081347E347E347E34BD34FF34FF340A10A4
:100020008A100A11820700347E347E347E34813493
:10003000FF34FF340A108A100A1182070034763424
:1000400076347E347E34FF34FF340A108A100A116D
:1000500082070034F634F634FE34FE34FF34FF34C5
:100060000A108A100A11820700347F347F347F34EB
:100070007F34FF34FF340A108A100A118207FE34DD
:10008000FE340034FE34FE34FF34FF340A108A108C
:100090000A118207FF34FF34FF34FF34FF34FF348A
:1000A000FF342330840083130008031968280130CB
:1000B000F800BF30F7006400F70B5B28F80B5928F5
:1000C0004A30F700F70B622800006400800B5728C5
:1000D0000034840183131F30830583161F149F147B
:1000E0001F159F1107309C00FF308312A00083165C
:1000F0001F109F141F159F151F1383121F179F1387
:1001000083169F1383121F148316091283129412ED
:10011000A012200883168700831220162008831659
:1001200087008312A01120088316870001308312F4
:1001300094000030831694000108C7390838810004
:10014000831290010030F800920000308316920074
:1001500007309C00050864000230F700F70BAE285A
:10016000B1281C0883120D1383169D010030F8007E
:1001700083121F08C73978049F0064000230F7001B
:10018000F70BC028C3281F151F19C4281E08A2007A
:1001900022080A3C03188029A1012108063C031CFF
:1001A000DE2821083020A30083168601831223084D
:1001B00086000130A3005120A10ACD28A101210809
:1001C000063C031CF02821081A20A3008316860190
:1001D0008312230886000130A3005120A10ADF28E2
:1001E000A1012108063C031C022921080F20A300BD
:1001F000831686018312230886000130A300512054
:10020000A10AF128A1012108063C031C1429210898
:100210004620A3008316860183122308860001303E
:10022000A3005120A10A0329A1012108063C031CB7
:10023000262921081A20A300831686018312230889
:1002400086000130A3005120A10A1529A10121082F
:10025000063C031C382921082520A30083168601AB
:100260008312230886000130A3005120A10A272908
:10027000A1012108063C031C4A2921082520A300CE
:10028000831686018312230886000130A3005120C3
:10029000A10A3929A1012108063C031C5C29210877
:1002A0001A20A300831686018312230886000130DA
:1002B000A3005120A10A4B29A1012108063C031CDF
:1002C0006E2921080420A3008316860183122308C7
:1002D00086000130A3005120A10A5D29A101210857
:1002E000063C031C802921083B20A30083168601BD
:1002F0008312230886000130A3005120A10A6F2930
:04030000C3286300AB
:02400E00393F38
:00000001FF
